:020000020000FC
:100000000FC0F2C0F2C0F4C0F4C0F4C0EFC0EFC043
:04001000F3C0F1C088
:10002000F89400E811E006BD16BD0FE90DBF00E32E
:1000300008BB00E107BBB0E0A0E6D0E0C0EA00E00A
:100040000D93BD17E9F7AC17D9F700E805BF00E03D
:1000500004BF00E005BD00E002BF00E00FBD05E009
:1000600003BF00E006BF00E009BD00E008BD00E2FC
:1000700007B907E006B900E003B900E004BB00E8F7
:1000800008B909E3102F177F01BD11BD00E00BBFB8
:1000900000E005BB00E009BF00E60ABF0EE008BFB4
:1000A00000E0E02E90E07894A895C49A06B30095FD
:1000B0000F70003021F420E010E00AE05AC0013057
:1000C00021F420E010E00EE154C0023021F420E0E1
:1000D00010E00CE34EC0033021F420E010E008E70C
:1000E00048C0043021F420E011E00CE242C00530A9
:1000F00021F420E012E008E53CC0063021F420E0C5
:1001000017E008E036C0073021F420E01EE000E1EF
:1001100030C0083021F420E01CE100E22AC00930A0
:1001200021F420E010E000E024C00A3021F420E0B7
:100130001CE800EA1EC00B3021F421E011E500E8C4
:1001400018C00C3021F422E013EA00E012C00D3098
:1001500021F426E017E900E80CC00E3021F42DE070
:100160001FE200E006C00F3021F427E21DE800E0A6
:1001700000C030E00894030B130B230B49E050E060
:1001800060E0A8956A95E9F75A95D1F74A95B9F7CD
:10019000203079F7103069F7003059F700E003BFDD
:1001A00000E00FBD00E003BF00EC03BFC49800E017
:1001B00006B900E007B900E808B903E000BF02E0B3
:1001C00000BF03E005BD01B5086101BD077F01BDAA
:1001D00005B7077E006105BF006205BF03E012E0BE
:1001E00000BF10BF889560CF189518951895189581
:1001F000189518951895189518951F932F932BE11E
:100200001EE11A95F1F72A95D9F70A95C1F72F91B2
:040210001F9108959D
:00000001FF
